:1000000012C0189518951895189518951895189563
:100010001895189518951895189518951895189578
:100020001895189518958FED8DBFC0ECE8EB4E2E06
:10003000DD275D2EEEE7F0E0A0E6B0E088278D93A7
:100040003197E9F766248FEF87BB8C9A8D9A8E9A49
:100050008EE180936C008FEF88BB80E782BB7DD000
:1000600088EE93E0A1D1E6E6F0E0FA93EA937CD043
:100070002296A6E68C9183508C9381E090E0A4E6D2
:100080008D939C93A4E60D911C910A3F50E01507B7
:1000900010F009F061C000916600003081E008F4C2
:1000A00080E08F9300916600033681E010F009F044
:1000B00080E09F918923882309F407C0E6E6F0E0F9
:1000C000FA93EA9363D0229643C000916600043607
:1000D00081E008F480E08F93009166000F3781E0A3
:1000E00010F009F080E09F918923882309F402C071
:1000F0000CD12EC000916600003881E008F480E049
:100100008F9300916600053F81E010F009F080E0D8
:100110009F918923882309F402C0F7D019C0009168
:100120006600063F81E008F480E08F93009166004E
:100130000F3F81E010F009F080E09F918923882330
:1001400009F406C0E6E6F0E0FA93EA938ED0229630
:10015000A4E61BD108F096CF86CF5DD110E972D10D
:100160001EEE70D166D1089556D110E96BD11AEA0E
:1001700069D15FD150D111E965D183D1A881B9810D
:100180001C937DD1A7E61C9354D10895009167007C
:10019000003009F004C080E08093610003C085E076
:1001A00080936100ECE7F3E0A1E68C919927A0E64B
:1001B0001AD180E482BBA0E68C9188BB85E090E0F8
:1001C000F3D0A881B9810C914AE010D1A1E68C93BB
:1001D000ECE7F3E0A1E68C919927A0E604D180E258
:1001E00082BB0091600040E8040F08BB85E090E00E
:1001F000DBD0A881B9810C914AE0F8D0A1E60C933C
:10020000ECE7F3E0A1E68C919927A0E6ECD080E141
:1002100082BB00916100013008F003C080E088BB20
:1002200003C0A0E68C9188BB85E090E0BDD080E063
:1002300082BB40916C0000916600041710F009F039
:1002400001C012C081E080936300009163000A3016
:1002500010F009F009C08FE090E0A6D0A3E68C91E1
:100260008F5F8C9308F4F1CF089500E0A881B981E5
:100270004C91041BABE60C93ABE68C9181508C93B4
:1002800000916700003009F004C085E080936100B0
:1002900003C080E080936100ECE7F3E0A1E68C917D
:1002A0009927A0E6A0D080E482BBA0E68C9188BB11
:1002B00085E090E079D000916B004AE097D0A1E60C
:1002C0008C93ECE7F3E0A1E68C919927A0E68BD024
:1002D00080E282BB0091600040E8040F08BB85E02B
:1002E00090E062D08AE080936100ECE7F3E0A1E661
:1002F0008C919927A0E677D080E182BBA0E68C9113
:1003000088BB85E090E050D008958AE0809361003A
:10031000ECE7F3E0A1E68C919927A0E664D080E4B5
:1003200082BBA0E68C9188BB85E090E03DD08AE05E
:1003300080936100ECE7F3E0A1E68C919927A0E6B9
:1003400052D080E282BBA0E68C9188BB85E090E031
:100350002BD08AE080936100ECE7F3E0A1E68C917A
:100360009927A0E640D080E182BBA0E68C9188BBB3
:1003700085E090E019D00895F894FFCF3F065B4FD9
:10038000666D7D077F6F40803846ED91FC91319618
:10039000FC93EE9308953197F1F70895689462F80D
:1003A0000895E89462F80895EF93FF93EE27E82B01
:1003B000E92B31F0E4ECF9E03197F1F70197D1F74F
:1003C000FF91EF910895C89531960020089591E02E
:1003D00005C092E003C094E001C098E0F4DF0D9204
:1003E0009A95E1F70895E80FF91FF1CFFF93881B65
:1003F000F9E0001FFA9511F4FF910895881F841BFE
:1004000018F4840F8894F5CF0894F3CF91989098BE
:10041000899888980895889A899803D0889801D0F7
:10042000899AEF93FF93E9E0F0E0B5DFFF91EF9158
:100430000895889A899AF5DF8898809BFECFF1DF2E
:100440008998EFCF0894111F01C0110F69F0889AA5
:1004500018F40000899802C0899A00C0E2DF8898E9
:10046000809BFECFDEDFF1CF889A8998DADF88980B
:10047000809BFECFE8948199689462F8D2CF08946B
:1004800001C08894331F11E0889A8998CADF889840
:10049000809BFECFC6DF889481990894111FA0F736
:1004A000889A379510F4899801C0899ABADF88989C
:0804B000809BFECFB6DF08952A
:00000001FF
